:020000020000FC
:10000000ABC949C20000000025C000004FC100007C
:10001000000052C1000000000000000002030406BE
:10002000080C101820304060800002030406080C01
:10003000101820304080FF000406080C10182030F3
:10004000406080A0C0000D0D0405060D050D0603DF
:10005000030302004FB662FD1EC070FF1AC165FDAA
:10006000FAC00994C0919700C395C0939700C5E06A
:10007000C519B8F3D0919700CD1B98F3C8E7089441
:1000800083FDC795C4BDC52DCC2321F4C0E083FDFD
:10009000C0E8C4BD09C171FF03C0909A949A959AB3
:1000A000C52D089483FDC795C4BDC09399006B7F8F
:1000B000C52DCF3F09F443C0C0919800C395C093AC
:1000C000980070FF37C082FD05C0909A949A959A67
:1000D0004FBE18957860C091A000CC2391F0C091DC
:1000E0009800CA95D091A000CD1B58F0777FC091A1
:1000F0009800D0919F00CD1B08F41CC0209298005E
:1001000019C0909A949A959AC5E0CA95F1F7C09152
:100110007500CA95C2FD09C0C1FD05C095FF979A3B
:1001200095FD919A0EC0939A0CC095FF919A95FDFA
:10013000979A07C0909A949A959A4FBE18952092D4
:1001400099004FBE1895A5C0552021F095FF9098B5
:1001500095FD9598949A9DC0552009F0949895FF27
:10016000959A95FD909A95C0552021F095FF959808
:1001700095FD909895FF909A95FD959A8AC095FF68
:10018000919895FD979895FF979895FD9198C5E062
:10019000CA95F1F7552021F095FF909895FD959817
:1001A000949A77C095FF919895FD97989398C5E09C
:1001B000CA95F1F7552021F095FF909895FD9598F7
:1001C000949A67C0939895FF919895FD9798C5E08C
:1001D000CA95F1F7552009F0949895FF959A95FDE9
:1001E000909A57C0939895FF979895FD9198C5E080
:1001F000CA95F1F7552009F0949895FF959A95FDC9
:10020000909A47C095FF979895FD91989398C5E06F
:10021000CA95F1F7552021F095FF959895FD909896
:1002200095FF909A95FD959A34C095FF979895FD06
:10023000919895FF919895FD9798C5E0CA95F1F72B
:10024000552021F095FF959895FD909895FF909AEF
:1002500095FD959A1EC082FF1CC0C0917500C2FD1D
:100260000BC0C1FD11C095FF919895FD979895FF22
:10027000979895FD91980DC0C1FDF5CF95FF919888
:1002800095FD9798939805C0939895FF979895FD3D
:100290009198C52DC095089483FDC795C4BDC093A2
:1002A00099002092970064604FBE18954FB6C0E148
:1002B000C8BF6E7F4FBE18953FB68F7EABB7A07498
:1002C000A2118061A0E0ABBFA9B7AE7FA9BF7894AF
:1002D000A0916600AA2349F0A92FAF7151F1A09116
:1002E0006600AA95A093660024C040E050E0A0B349
:1002F00096FFA095A2FD4FEF96FDA3E096FFA2E02A
:10030000A5BFAA27A064AABF8D7FA0B396FFA09522
:10031000A2FD5FEF451749F7A8E161FDA0936600D4
:10032000A92FAF7119F0A8E1A093660040938D004A
:100330008160A0916700AA2331F0A0916700AA957F
:10034000A093670007C0A92FAF7121F08061AA2791
:10035000A064AABF80FF4BC0A0918D004A2F8E7F62
:10036000A92FAF71E1F0A091AE00A430C1F4403FDD
:1003700008F040EFA42FA295AF704A0F5091B00043
:10038000533069F0A695A69550FD01C0A69552FD83
:1003900003C0A41B4A2F03C04A0F08F44FEF409339
:1003A000610071FF08C0A091610050919200A517F3
:1003B00010F0509361004091AE00443029F5A091B7
:1003C000610040916300A41B70F04091CF00A40B2A
:1003D00050F0A0916300A40FA093630040F4AFEF2E
:1003E000A093630004C0A0916100A09363004091BA
:1003F0006300A09192004A1708F04A2FA091940040
:100400004A1708F04A2F542EA52DA03408F0686032
:10041000A0916000A395A093600051F0F894A9B753
:10042000A160A9BF84FF02C0A0E4ABBF3FBE189586
:1004300041E050916600552331F0A92FAF7119F4B6
:100440005A9550936600A0918D00A13018F020922B
:1004500090000DC02092910020929A00A0919000EF
:10046000AF5FA093900018F0AFEFA0939000A09121
:100470009300A65F20F05FEF5093930002C0A0931B
:100480009300F894A9B7A160A9BF84FF02C0A0E4BB
:10049000ABBF3FBE18953FB64CB55DB58F7EABB7D1
:1004A000A074A2118061A0E0ABBFA9B7AE7FA9BFC5
:1004B000789481FD26C096FDA2E096FFA3E0A5BF3B
:1004C0008260A0B396FFA095A2FF05C04093640090
:1004D0005093650033C196FDA3E096FFA2E0A5BF4F
:1004E000AA27A064AABF8D7FA92FAF7109F417C1F5
:1004F00040E0A0B396FFA095A2FD11C140938D00EE
:1005000004C196FDA3E096FFA2E0A5BF8D7F61FF29
:100510006BC096FDA2E096FFA3E0A5BFAA27A0644A
:10052000AABF82604093880050938900A090860003
:100530004A19B09087005B09BB24A2E0EA2EA22CE6
:10054000483CA0E05A0730F4A0E1BA2EE22CAAE021
:10055000AA2E27C04836A1E05A0730F4A8E0BA2EE8
:10056000E22CAFE0AA2E1DC0403DA2E05A0730F4B5
:10057000A4E0BA2EE22CAEE1AA2E13C0403AA5E0C8
:100580005A0730F4A2E0BA2EE22CACE3AA2E09C03E
:100590004839A8E05A0728F4A1E0BA2EE22CA8E7CF
:1005A000AA2EC42EA0918A00CA1AD52EA0918B0023
:1005B000DA0ADD202AF4AFEFC094D094CA1ADA0A1E
:1005C00020928C00CA14DE0418F4A1E0A0938C00E1
:1005D00040938A0050938B0040918800509189008D
:1005E0004093860050938700A09164004A1BA0911D
:1005F00065005A0B94FD7CC093FD7AC092FD76C0D5
:100600005695479591FD72C05695479590FD6EC0E1
:10061000D52EC42ED694C79461FD0CC0AC2DAC5120
:10062000AD2DA24008F07BC0DD2021F4AC2DA85CEC
:1006300008F475C0A0E0EA2E97FD08C0E090C20063
:10064000A091B400A33011F4E090CA00AAEFEA0E22
:10065000F22CF21CCE18DF084FB74170A091B40005
:10066000A330A9F4442329F095FD11C0F8949062B9
:1006700004C095FF0CC0F8949F7D909A949A959A27
:1006800091989398979871FD01C06068789444237D
:1006900069F0A091B400A33031F4AFEFC094D094CE
:1006A000CA1ADA0A03C040E050E022C0A091B400A8
:1006B000A33049F4CC0CDD1CA5E0CA1AD20818F40A
:1006C000A0E0CA2ED22CAFEFCA16D20418F04FEF1A
:1006D00050E00EC0F090A700CF9C412D000C441FAD
:1006E00050E008F012C04FEF50E00FC0569547950C
:1006F00094FF07C0552309F04FEFA42FA6954A0F8A
:10070000521D4F3F520508F04FEF40938D0081601E
:1007100061FF05C0AFE1A095A923AB299A2FA8E1FD
:10072000A0936600A92FAF7119F4AAE0A093660008
:1007300061FD04C0A92FAF7109F08F7EA6E0A093E0
:100740006700A92FAF7119F4AAE0A0936700F8948D
:10075000A9B7A160A9BF84FF02C0A0E4ABBF3FBEA0
:10076000189511E00AC013E008C01AE006C01EE1A7
:1007700004C014E602C018EC00C005E1BB27BA951E
:10078000F1F70A95D9F71A95C1F708952AE338E7E2
:1007900009C020E33CE806C02AE234EB03C025E2AE
:1007A00038EC00C0652CB1E05B2E12E095FD9F7D1A
:1007B00095FF9062BB279398BA95F1F7552009F001
:1007C0009498BA95F1F7949ABA95F1F7939ABA95E5
:1007D000F1F7552021F095FF909895FD9598B091EF
:1007E000A800BA95F1F795FF909A95FD959AB7E80C
:1007F000BA95F1F71A95D1F6022FB22FBA95F1F703
:100800000A95D9F73A9571F69398562C0895221BBC
:1008100039E0001F3A9509F40895221F211B18F4AE
:10082000210F8894F6CF0894F4CF622C722CB0E09C
:100830008894B395221F331FE0F737952795889446
:10084000912E802E020B130B10F4192D082D10F48D
:10085000889401C00894661C771CBA9571F7172D0F
:10086000062D0895322D11232AF43A9500951095FE
:10087000031B130BF894029F712C002D129F912CD7
:10088000802C7894780C172D921C292DB4E06B2EB7
:100890002695179507956A94D9F7332321F000958B
:1008A0001095031B130B08950091AE000430A1F1C5
:1008B000B0918D00B15008F010C0B0916100B093BC
:1008C0006300209277002092780020927900209295
:1008D0007A0020927B006F7B1FC06090AE00606446
:1008E000B0916100B093620008E317EC20917300AF
:1008F0003091740036952795B62DBA9541F036950E
:100900002795B62DBA95BA9511F0369527958DDFB6
:100910000093770010937800089566FF1BC0009144
:100920007700B09162000B1B10917800120928F437
:100930000038BFEF1B0740F009C00F37120508F45D
:1009400005C00FE710E002C000E81FEF00937C0035
:1009500010937D00089566FF39C000917C00B0912E
:1009600079000B0F10917D00B0917A001B1F20E0E1
:1009700030917D0033230AF42A95B0917B002B1F20
:100980001AF4203F40F00AC02F3008F407C00FEFE0
:100990001FEF2FE003C000E010E020EF3091630074
:1009A000B09192003B1718F4332331F009C0B09195
:1009B0007D00BB235AF004C0B0917D00BB2332F40C
:1009C0000093790010937A0020937B00089566FFCE
:1009D0002FC02091CD0000917C00000F10917D0070
:1009E000111F40DF11232AF40038BFEF1B0740F02E
:1009F00009C00F37120508F405C00FE710E002C068
:100A000000E81FEF002352F0B0916200B01B0B2FE3
:100A100018F0013008F00AC001E008C000950F5F2F
:100A2000B09162000B0F08F001C00FEF00937E0041
:100A3000089566FF2DC02091CE0000917A0010919C
:100A40007B0010DF11232AF40130BFEF1B0740F0B9
:100A500009C00F3F120508F405C00FEF10E002C0F7
:100A600001E01FEF112352F0B0917E00B01B0B2F5D
:100A700018F0013008F00AC000E008C000950F5FD0
:100A8000B0917E000B0F08F001C00FEF00936300E0
:100A900008950FEF677FB72FB670E9F46860B091E3
:100AA0007400B83008F0677FB0917400A1F00FEFC8
:100AB00010917400ACDEF894B09170000B9F112D72
:100AC000002D7894112309F00FEFB09195000B17CA
:100AD00010F4009195000093940008951ED374FFC4
:100AE000B7E074FDB7E0B068B064B7B9B6B1B0684C
:100AF000B064B6B936DE74FFB7E074FDB7E0B06835
:100B0000B064B7B9B6B1B068B064B6B9B6B1B6FD45
:100B1000FDCF04B115B1B6B1BF77B6B943D324E365
:100B20002093A30030E03093A400732E7694622EBD
:100B30006694620E731E262D372D0217130778F068
:100B40008090A300B4E3B80DB093A3008090A400FC
:100B5000B0E0B81DB093A400260D371DEECF8090F5
:100B6000A3009090A4001091A40016950091A300FA
:100B7000079516950795B091A300B00FB093A1000B
:100B8000B091A400B11FB093A20023E01695079581
:100B90002A95E1F72091AF002A9529F42092A3002D
:100BA0002092A4000AC02A9521F0800E911E2A9559
:100BB000E1F78092A3009092A40008952091AF00E5
:100BC000B6B1B6FDFBCF04B115B1B6B1BF77B6B9BA
:100BD000B091A500B395B093A500B83060F1209214
:100BE000A500B091CC00BB2321F1112329F0B091D5
:100BF000A600BF3F61F009C0B091A6000B1739F005
:100C000020F4BB2321F0BA9502C0B395E1F3009123
:100C10009200B093A600B03050F400ECB03038F43D
:100C200000E8B03020F400E4B03008F400E00093B5
:100C300092007F7E0895213099F00F3FB3E01B07AB
:100C400078F4B091A3000B17B091A4001B0740F4F7
:100C5000B0919200BB23A9F0BA95B093920011C055
:100C6000B0919200BF3F69F0B395B0939200B091FC
:100C7000B400B33031F4B0919200BC5F10F4B09383
:100C8000920000919200B0916300B01B10F40091AB
:100C90006300B09193000B1750F000919300B09156
:100CA0009300BF3F21F0B0919300B0939200B091B8
:100CB000AE00B43009F406C0B09194000B1708F0F0
:100CC0000B2F502EB091A500B73009F47061089534
:100CD00002E3F894B091D0000B9F012D000C001F8F
:100CE0007894B09192000B1710F00091920000934D
:100CF000610000936300502E0093950008952092A8
:100D00007300B8E0B0937400089520918000309192
:100D10008100F8940CB51DB5200F311F3BBD2ABDD5
:100D20006160B0E1B8BF7894209171003091720099
:100D30000093710010937200021B130B209173003B
:100D400030917400622E732EB4E08B2EB2E09B2E95
:100D5000B0917400B43010F08A949A94B83010F0C6
:100D60008A949A94769467948A94E1F726193709BD
:100D7000992021F0169507959A94E1F7200F311FDD
:100D8000209373003093740008F00895BFEFB09380
:100D90007300B09374000895209182003091830015
:100DA000F8940CB51DB5020F131F1BBD0ABD616081
:100DB000B0E1B8BF7894089560FDFECFEDDF0895EF
:100DC000B091BE0000916E00023808F0B395003A71
:100DD00008F0B395B63008F0B5E09B2EBCE08B2E42
:100DE000B0917400B33030F48394839482FF02C0D6
:100DF00083948394B23030F48394839482FF02C04E
:100E00008394839471FF03C0B3E09B2E822C1091D6
:100E100074000091730024E0169507952A95E1F778
:100E20000819120928F0B02FB250B12FB20910F4EE
:100E300002E010E0312F202F712E602E76946794FF
:100E4000B92DB330E9F0B0FD05C0060D171D262DF4
:100E5000372D06C0000F111F0250120922E030E0AA
:100E6000B92DB33068F0209384003093850000934F
:100E70008000109381006092820070928300089538
:100E800000938400109385002093800030938100AC
:100E90006092820070928300089560FDFECF2091E1
:100EA0008200220F30918300331FB72FB67021F0DC
:100EB0002091730030917400F8940CB51DB5020FA9
:100EC000131F1BBD0ABD6160B0E1B8BF78940895DF
:100ED00060612092760020E004C06061209276007C
:100EE00020E2B72FB67009F06F7E789460FD05C0E0
:100EF000B0917600BB2309F0089501E063FF0AC0BA
:100F0000B0917400B33008F002E0B0917400B630D4
:100F100008F003E071FF01C006E060FD06C0B0917B
:100F20007600BB2311F0789408951AE083FF1AE04D
:100F3000789400000000F89462FD03C014E183FF80
:100F400014E171FF01C018E7B4B530919900B31BEB
:100F5000B10B18F3B0917600B395B0937600B5E07D
:100F60003B2F6B2E722CB8B1B072B21709F073948C
:100F70003A95C9F77394761488F464FFB2CF6F7E04
:100F80003CB56DB47090730080907400370D681C90
:100F90006BBC3ABD6160B0E1B8BFA3CF64FDA1CF27
:100FA0000A9509F0BACF7894089571FF0AC0B091FC
:100FB0006D00B395B0936D0060FD0CC020926D0084
:100FC00009C060FD07C064FD05C067FD03C0BF9197
:100FD000BF916FC408952091840030918500F894EA
:100FE0000CB51DB5020F131F1BBD0ABD6160B0E13A
:100FF000B8BF78940895EFDF00E063FF03C064FF9B
:1010000001C001E0F89410916E00B7E01B9F212D04
:10101000102D7894200F26951795269517952695CF
:10102000179510936E00183718F4B8E7B0936E0058
:1010300000916E00B0916F000B1720F06062909AE3
:10104000949A959A60FDFECF0895F894919893989C
:10105000979882FF07C0E2E0F1E073FF03C0B5E0BC
:10106000BA95F1F795FF919A95FD979AB2E0B093F2
:10107000750089C0F89495FF959A95FD909A82FF26
:101080000DC0E2EFF0E073FF0BC0939895FF9798C7
:1010900095FD9198B5E0BA95F1F702C0ECEAF0E061
:1010A00062FF03C0552009F09498B3E0B093750037
:1010B0006AC0F89491989398979882FF07C0E2EEDF
:1010C000F0E073FF03C0B5E0BA95F1F795FF979A8A
:1010D00095FD919AB4E0B093750055C0F894949A38
:1010E00082FF0DC0E2EDF0E073FF0BC095FF919819
:1010F00095FD97989398B5E0BA95F1F702C0E4EAA8
:10110000F0E062FF06C0552021F095FF909895FD14
:101110009598B5E0B093750036C0F894919893987F
:10112000979882FF07C0EFEBF0E073FF03C0B5E0D4
:10113000BA95F1F7939AB6E0B093750024C0F8948D
:1011400095FF909A95FD959A82FF10C0E5E1F1E038
:1011500073FF0EC095FF919895FD979895FF97980E
:1011600095FD9198B5E0BA95F1F702C0E4EBF0E097
:1011700062FF06C0552021F095FF959895FD909847
:10118000B1E0B093750067FF0AC00CD0B5E0BA9526
:10119000F1F7B5E0BA95F1F7919A939A979A6F7D26
:1011A0007894089523EA30E0F901909A949A959AF8
:1011B0009198939897986B7F0895ACEAB0E009E016
:1011C0000D9309E00D9304E00D9301E00D9303E00E
:1011D0000D930FEF0D9309E00D9301E00D9301E0E6
:1011E0000D9301E00D93A8EBB0E001E00D930FEF3C
:1011F0000D930D930FEF0D930D930D9303E00D934E
:1012000006E00D930FEF0D930D9305E20D9300EDA6
:101210000D9308E20D9300E50D9304E00D930DE0AE
:101220000D9302E00D9300E00D930AE70D930FEF8D
:101230000D9301E00D9308952091BF0009E011E0A6
:10124000223011F405E011E0233011F405E012E042
:10125000243011F405E013E0253011F409E017E023
:10126000263011F400E010E000939F001093A000DE
:101270002091B3008B7F233009F48460777F233083
:1012800009F47860B091B400B33019F09F7DB1FDDE
:1012900090629F7BB091B500B1FD9064B22FB230E7
:1012A00011F0886001C0877F0895ECE1F0E00091C3
:1012B000AC000A95E00FF21DB491B093CD000091FF
:1012C000AD000A95E00FF21DB491B093CE006ADF35
:1012D0000895EAE2F0E00091C7000A95E00FF21DE0
:1012E000B491B093CF005EDF0895E8E3F0E00091A1
:1012F000B2000A95E00FF21DB491B093D00052DF16
:1013000008950895B091C8000FEF1CE0B23011F4B9
:1013100000EA1AE0B33011F402E815E000936F0020
:1013200010937000089508952091C2003091C30079
:1013300097FF02C020E03FEFB32FB21B6B2EB258D5
:1013400010F4B2E86B2E00E00395609EB12DB0580A
:10135000D8F30093A7000895F894E3E0F0E0B9E033
:10136000B7BFB491B078C1F3F894A895B1B5B8619E
:10137000B1BDB0E0B1BDB4E0BEBFBFE5BDBF12DFDF
:10138000B4E0B8BBB4E1B7BBB0E0B5BBB0E0B4BB50
:10139000B1E3B2BBBBEBB1BB2224A0E0B0E02D9225
:1013A000AA31E9F7A0E6B0E00FEF2D920A95E9F730
:1013B00004DF9FD241DF79DF8CDF97DFA2DFA2DF7E
:1013C000B2DFB2DF0091C4000093A800EBDEB2E010
:1013D000B3BFB2E0BEBDB2E0B5BDF894CCD9D6D9AA
:1013E000C6D9D7D9C4D9D8D9C2D9C5D9C4D9C1D9F0
:1013F000B1E5B8BFB9BFB0B7B860B0BFB6B1B460FF
:10140000B6B9AFD978946ADBB0E4BBBFBB27B06490
:10141000BABF8D7FB0D9B1E0B0936900626025E0BA
:10142000B0918C00BB2309F425E09DD9B0918D00CB
:10143000B230A8F3B92FBF7100918F0000938E00D6
:10144000B0938F00B01759F72A9551F76D7F96FD2D
:10145000B3E096FFB2E0B5BFBB27B064BABF8D7FE3
:1014600088D981D902E0B92FBF7109F400E0B091A9
:101470008D00B017B0F3F89489D988D987D97894BA
:101480007AD920927F00B091B400B33009F472C0D1
:101490006AD9B091B800B13008F46CC0B09169005D
:1014A000B13008F467C0B92FBF71C1F0B0918D00A1
:1014B000BF3F08F45FC0F89472D978945AD9B091BC
:1014C0008D00B130C0F7F89461D94FD95FD97894C5
:1014D00050D9B0918D00BF3FB0F3D4C2B3E09B2E82
:1014E0009068F89421DF789444D9F8949F771CDFB2
:1014F00080908D00B0918D00BF37789408F442C081
:1015000030D9F8944CD978949A9451F7B82DB550B5
:10151000B093C30030D9F89419D287D27894BAE046
:101520009B2E9068F89400DF789423D9F8949F77E5
:10153000FBDE80908D00B0918D00BF37789478F7F6
:1015400010D9F89423D911D921D978949A9449F7CC
:10155000B82DBB5FB093C2000ED9F894F7D174D206
:10156000789407D9F894E0DE7894B0918D00BF3F6D
:10157000C0F388C200918D00B0917F000B1710F06E
:1015800000937F00F6D801E0B091B400B35009F4A5
:1015900005E0B0918D00B01708F075CFF894FFD832
:1015A000FED8FDD87894E7D82092690020926A008E
:1015B00020926B00B0916A00B395B0936A00BF3F70
:1015C00069F5B0916B00B395B0936B00B091C60014
:1015D00009E1BA9559F002E3BA9541F00DE7BA95E1
:1015E00029F00AEFBA9511F020926B00B0916B00D0
:1015F000B017A0F0B0916B00BA95B0936B00B4EB4C
:10160000B0936A00B091C500B093A800F894C7D811
:101610007894B091C400B093A800ABD8A6D8B0918C
:101620006600BB2321F4B92FBF7109F4F7CEB09146
:101630008D00B63008F4BECFB091B400B35009F0BD
:1016400098D8B0916600BB2309F4E8CEF894AADDDF
:10165000209261002092620020926300522C7894C4
:10166000B091B100B093960020927700209278005C
:101670002092790020927A0020927B002092A5008F
:1016800060E070E020926E003ADBB8E0B093A50015
:10169000706167D874FFB7E074FDB7E0B068B064FC
:1016A000B7B9B6B1B068B064B6B9B6B1B6FDFDCFE2
:1016B00004B115B1B6B1BF77B6B9112309F00FEF78
:1016C0000093A6007BDAB8E0B093A500706180902B
:1016D000B300B2E0B093B300AFDD8092B300F894F2
:1016E000BFEFB0939200F4DAB0916100B093920032
:1016F000B0939300B09394007894B1E0B0936100FC
:10170000B09363005B2EB0939B00B0919100B093B7
:101710009A007160726020926D00FFDC10DDF5DAD6
:10172000EEDA4EDB04C088DD2092A5007F7E95FFB7
:10173000B4E095FDB2E0B068B064B7B9CEDB35DC9B
:101740004ADCB2D858DC81DCE0DA36DB39DBA5DBF9
:10175000B3E0B068B064B7B9BBDB27DC3CDCDDD8F4
:1017600098D949DC87DCD1DA27DB2ADB96DB95FFC9
:10177000B2E095FDB4E0B068B064B7B9AEDB15DC9B
:101780002ADCE9D838DC95DCC0DA16DB19DB85DB2E
:1017900095FFB4E095FDB2E0B068B064B7B998DBEE
:1017A00004DC19DC14D927DC99DCAFDA05DB08DBB3
:1017B00074DBB3E0B068B064B7B98FDBF6DB0BDC89
:1017C00038D919DCAADCA1DAF7DAFADA66DB95FF98
:1017D000B2E095FDB4E0B068B064B7B979DB74FFEE
:1017E000B7E074FDB7E0B068B064B7B9B6B1B0683F
:1017F000B064B6B9DADBEFDBFEDBA1DC86DADCDA7B
:10180000DFDADCD94ADB71FF2EC067FD2CC0B09156
:101810009500B0939200B0939300B0919100B09373
:101820009A00B1E0B0939B0014E624E1B0916D0002
:10183000B11798F07D7F746020936C00B091B40074
:10184000B33051F4B0919500B0939200BFEFB093D4
:101850009300B0E2B093940006C0B0918D00B13017
:1018600008F065CF26C072FF10C067FD0EC0B091B2
:101870006C00BA9511F47B7F56CFB0936C00B09199
:101880008D00B13008F053CF14C0B0919000BA3F32
:1018900080F4B92FBF7121F4B0916600BB2349F0E9
:1018A000B091740000EF67FF01C000E6B01708F4C4
:1018B0003ECFF89477DC8090B300B2E0B093B300F1
:1018C000BBDC8092B30020926100209262002092E3
:1018D0006300522C209296007E7F789442D762DC7F
:1018E000B92FBF7129F4B0916600BB2309F496CDDE
:1018F0005DCEEDE0F0E023D0053509F01BC0EEE051
:10190000F0E01DD00A3A09F015C03AE0ACEAB0E0C8
:10191000E3E0F0E014D00D9331963A95D9F735E134
:10192000A8EBB0E0EFE0F0E00AD00D9331963A95E5
:10193000D9F702C042DC0AD0E4E2F0E00895E19970
:10194000FECFEEBBFFBBE09A0DB308951ED03AE088
:10195000ACEAB0E0E3E0F0E00D910FD031963A95BB
:10196000D9F735E1A8EBB0E0EFE0F0E00D9105D05C
:1019700031963A95D9F712D00895E199FECF0DBB73
:10198000EEBBFFBBE29AE19A0895EDE0F0E00FEFC5
:10199000F4DFEEE0F0E00FEFF0DF0895EDE0F0E0CF
:1019A00005E5EBDFEEE0F0E00AEAE7DF08953091CD
:1019B000A9000091AA00313011F40093AC0032303C
:1019C00011F40093AD00333011F40093AE003430C5
:1019D00011F40093B000353011F40093AF003630AD
:1019E00011F40093B200373011F40093BE00383088
:1019F00011F40093C700393011F40093BF003A305E
:101A000011F40093B3003B3011F40093C8003C3054
:101A100011F40093B4003D3011F40093B500089523
:101A200025E0A9D62A95E9F70895B0D6B2D6B4D65E
:101A3000B6D69BD6ABD6ADD6AFD6B1D696D6A6D6B1
:101A4000A8D6AAD6ACD60895AAD6A6D6A2D69ED691
:101A50008CD6A5D6A1D69DD699D687D6A0D69CD60B
:101A600098D694D608958090A9009090AA008ED61A
:101A70008DD68CD67AD68A94D1F791D676D69A948A
:101A8000E1F70895F894D1DF7894CADFC9DFB1E0B7
:101A9000B093A900B1E0B093AA002092AB00F894F3
:101AA000E2DF7894B5E06B2E70908D0064D6B09133
:101AB0008D007B16C9F7B13018F0BF3F40F107C069
:101AC00076DFF89443DFB1DFB8E0B1BDA9DF6A94F7
:101AD00059F7B091AB00B395B093AB00B33008F4B5
:101AE000DECF9EDFB091AA00B395B093AA00F89420
:101AF000B091A900BA95E6E4F0E0EB0FF21D049175
:101B000078940395B091AA00B01708F4C6CF88DF87
:101B100087DFB091A900B395B093A900B091A90057
:101B2000BE3008F4B7CF49DBF89410DFB8E0B1BDA0
:021B300077DF5D
:00000001FF
